:100000000C942A001895000018950000189500001F
:10001000189500001895000018950000189500002C
:10002000189500001895000018950000189500001C
:10003000189500001895000018950000189500000C
:1000400018950000189500001895000018950000FC
:10005000189500008FE58DBFC0E2ECEA4E2E84E0DB
:100060008EBFD4E0F3E05F2EEEEFF3E0A0E6B0E069
:1000700088278D933197E9F76624899A9198889813
:100080008D9A8C988E9A9598AEE6B0E0EAEBFBE0FC
:100090000E940905A2E7B0E0EEEBFBE00E94090533
:1000A000E2E7F0E00E94E203EEE6F0E00E94DD030A
:1000B0000E944D04FF27EDE0A6E7B0E00E94D705BF
:1000C000E2ECFBE00E94B4020E94BC02E0EFFBE025
:1000D0000E94B402A4E9B3E0E6E7F0E00E94DD0389
:1000E0000E94F0020E94C0020E94BC02ECE6F0E016
:1000F000FA93EA930E94D5002296E4E0FCE00E9485
:10010000B402A4E9B3E0ECE6F0E00E9479050E94B5
:10011000C002EAE7F0E0FA93EA93ECE6F0E0FA9343
:10012000EA935A924A9281EF93E0A42DB52D8D93D4
:100130009C9382E00E94FA015A924A9289E290E0EE
:10014000A42DB52D8D939C9382E00E94FA01E6E7E1
:10015000F0E0FA93EA930E9427012A9684E00E9435
:10016000F601ECE0FCE00E94B402A4E9B3E0AF9336
:10017000BF93EAE7F0E00E94DD030E94F00211E085
:1001800001E0BF91AF910E941E05E4E9F3E0A4E90C
:10019000B3E00E94D2050E94C0020E94BC0284EF1C
:1001A00091E00E94E1020C94760000E010E020E073
:1001B00030E0AFE7B0E00D931D932D933C9381E0C9
:1001C00080937E0000917E00013018F011F00C94B5
:1001D0000C01ECE6F0E0FA93EA930E947401229697
:1001E000AFE7B0E00D911D912D913C91ACE6B0E0F0
:1001F0004D915C91662777270E946605AFE7B0E0D6
:100200000D931D932D933D93AEE7B0E08C918F5FDE
:100210008C9310F40C94E200AFE7B0E00D911D91C7
:100220002D913C9141E050E060E070E00E943E0280
:10023000AFE7B0E04D935D936D937D93AFE7B0E092
:100240008D919C91A881B9818D939C930895EC81A7
:10025000FD81D190E080FF2400270E9401040E94CC
:1002600032042F933F934F935F93EE81FF81D190A0
:10027000E080FF2400270E9401045F914F913F918D
:100280002F910E94A404FF27EDE0A3E8B0E00E94B4
:10029000D705E881F9810E94E203E3E8F0E00E94DB
:1002A000DD030E944D04FF27EDE0A7E8B0E00E94C7
:1002B000D705E7E8F0E00E94E203EA81FB81D190F4
:1002C000E080FF2400270E9401040E94B304FF275E
:1002D000EDE0ABE8B0E00E94D705EBE8F0E0A885E0
:1002E000B9850E94D7050895BB27A0E38C9184FBB4
:1002F000DEF388E090E00E94E102959A0027BB2798
:10030000A0E38C9184FB0EF401E041E0041710F0AF
:100310000C948C010C947E01959880E090E0A0E90B
:10032000B0E08D939C9381E080938F0000918F00CB
:100330000C3018F011F00C94E1019598BB27A0E364
:100340008C9184FBDEF388E090E00E94E10280E083
:1003500090E0A2E9B0E08D939C93969A959A00273D
:10036000BB27A0E38C9184FB0EF401E041E004176D
:1003700010F00C94C901A2E9B0E00D911C9141E08C
:1003800050E0040F151FA2E9B0E00D931C930C94EC
:10039000AF0195989698A0E9B0E00D911C91A2E963
:1003A000B0E04D915C91040F151FA0E9B0E00D93F2
:1003B0001C93AFE8B0E08C918F5F8C9310F40C9499
:1003C0009601A0E9B0E00D911C914CE050E00E9434
:1003D0002102A0E9B0E04D935C93A0E9B0E08D91DB
:1003E0009C91A881B9818D939C930895481A882780
:1003F000580A0895480E8827581E089500FC10D00A
:10040000089503D01ED001F8F9CF0024E89457FFD7
:1004100002C009D0689400F80BD010F801240895A8
:1004200002D009D00895509540954F5F5F4F0895D1
:10043000E89417FF0895009510950F5F1F4F68947B
:100440000895352F242FE894452B11F468940895CE
:10045000512F402F0027112780E1440F551F001F07
:10046000111F021B130B416018F4020F131F4E7F64
:100470008A9599F7089500FC05D0089530D005D0ED
:1004800001F8F9CF37D03FD00895842F952FA62FAC
:10049000B72FE894452B462B472B11F46894089509
:1004A000402F512F622F732F002711272227332728
:1004B000F0E2440F551F661F771F001F111F221FF8
:1004C000331F081B190B2A0B3B0B416028F4080F44
:1004D000191F2A1F3B1F4E7FFA9559F708950024D4
:1004E000E89477FF02C006D0689400F809D010F8AD
:1004F0000124089512D04F5F5F4F6F4F7F4F0895D3
:10050000E89437FF089500951095209530950F5F7A
:100510001F4F2F4F3F4F6894089540955095609519
:10052000709508953197F1F70895689462F80895E9
:10053000E89462F808958F939F9383E690E0019783
:10054000F1F79F918F91089580952AE090E00894AB
:1005500010F0919802C0919A0000EDDFECDF9695C3
:1005600087952A95A9F70895C895802D882319F0B5
:10057000EBDF3196F9CF08958DE0E6DF8AE0E4CF36
:10058000A4E9B3E08D91882311F0DEDFFBCF08955D
:100590008F939F9383E690E00197F1F79F918F915E
:1005A000089529E0809BFECFF3DFF2DFF1DF88942E
:1005B000809908942A9519F087959795F6CF80959C
:1005C0000895EF93FF93EE27E82BE92B31F0E0ED50
:1005D000F7E03197F1F70197D1F7FF91EF91089587
:1005E0008DE207FD8D938F2D881F802F881F8F57D9
:1005F000082F6894F7F8802F87FF15C080958395A2
:10060000082F80E38D938EE28D93802F815228F006
:1006100080E38D9399279C93089544270A95802F12
:1006200009F196D01FC0805230F09EE49D9381E482
:100630008D939D93EFCF4427DF92EF92FF920F931C
:100640008FE1801B11F0082F83D089D09EE29D930B
:100650000F91FF90EF90DF9044270395003209F44B
:10066000D7CF2BD03F93E0EFF6E038E12F2D1E2DB2
:100670000D2DFF24EE24DD244427000F111F221F1F
:10068000A8F42F923F920E940105102C0E940105B0
:10069000202C0E940105302C0E9401053197410D4C
:1006A000D21CE31CF01C3F902F9001C03396319672
:1006B0003A9519F73F9107D0AFCFDD0CEE1CFF1C28
:1006C0000A95D9F70895002719E058D08F93802B09
:1006D00011F0039501C08F911A95B9F7802F8823E7
:1006E00009F496CF8F91805D8D930A95D9F792CFBB
:1006F0000065CD1D80B2E60E40597307A0ACB9036A
:1007000050D6DC01286BEE0094357700CA9A3B0086
:1007100065CD1D00B2E60E0059730700ACB90300A9
:10072000D6DC01006BEE0000357700009A3B00003C
:10073000CD1D0000E60E000073070000B9030000A5
:10074000DC010000EE000000770000003B0000002C
:10075000F694E794D79447950A95D1F70895002722
:100760000DD08F9303958F2D8E298D29842BC1F762
:100770008F91805D8D930A95D9F74CCF1F930F937E
:10078000002710E2440FDD1CEE1CFF1C001F802F11
:100790009AE0890B10F0082F43951A9599F7802F4E
:1007A0000F911F910895D094E094F09491E0D90EA8
:1007B0009927E91EF91E10950895D190E190F190C6
:1007C0000191089521913191419151910895102FF6
:1007D00090E8FF0C001F0927990FF7941078652FF8
:1007E00090E8440F551F5927990F479560780038B6
:1007F0000895FF0C90E89027110F9795F794092F13
:100800000895102FBD2CDE2CEF2CF02E11234AF46E
:10081000B094D094E094F0949FEFB91AD90AE90A01
:10082000F90A0EE1FF2039F4FE2CED2CDB2CBB2461
:100830000850C2F766C032F00A95BB0CDD1CEE1CF6
:10084000FF1CF9CF01D0D5CFB7FE089590E8B916B7
:1008500011F4D0FE08959FEFD91AE90AF90A09F4B4
:1008600003950895502F2D2D3E2D4F2D612F089566
:100870002DEC3CEC4CEC5DE366270FC09EDFF2DF15
:10088000DD24EE2490E8F92E0FE307C09BDF05C0BE
:100890002227332740E251E46627552351F10023F4
:1008A00081F195DF71F11627005850580894050B17
:1008B00018F407FD03C025C007FD23C046953795F2
:1008C0002795F694E794D79422D0FF202AF0DD0CE8
:1008D000EE1CFF1C015073F09D2D969548F0DD2015
:1008E0003AF4EE202AF491E0D90E9927E91EF91E78
:1008F00080CF07C09FE7092FF92A9FEFD92EE92E55
:100900000895DD24EE24FF240027112708959F92E7
:100910009924AA24BB2488E1D216E306F40628F021
:10092000D21AE30AF40A089401C08894991CAA1CFC
:10093000BB1CDD0CEE1CFF1C8A9571F7D92CEA2C30
:10094000FB2C9F9008953EDF42DF503829F090E85D
:1009500069270CC00AF045D04CCF5FE3222733272C
:10096000442701C02FDF33DF5038B1F3003899F34B
:10097000902F951B8BF312F434D0FACF983118F0E6
:10098000222733274427983028F0232F342F442759
:100990009850F9CF992329F04695379527959A9540
:1009A000D9F7912F962742F014D0B0F6F794E79438
:1009B000D7940F5F8BF69ECF10D051F008F4F3DE82
:1009C000FF2052F2DD0CEE1CFF1C0150CBF792CF42
:1009D00098CFD20EE31EF41E0895D21AE30AF40A49
:1009E0000895DF92EF92FF920F931F93D22EE32E82
:1009F000F42E052F162F6F915F914F913F912F91FC
:100A00000895C89531960020089591E005C092E0C0
:100A100003C094E001C098E0F4DF0D929A95E1F7ED
:100A2000089599278D9193958823E1F793951196D1
:100A30008C9311978E919A95D1F70895EA2FFB2FF9
:100A400000244C918D9103948E32E1F711248D9105
:100A500013948823E1F71A94101640F41197202F6D
:100A60002119239580E38D932A95E9F7113039F503
:100A70009927AE2FBF2FA00DB91FA00FB91F8C91C2
:100A80009C93853308F421C031E08E918E32E9F3D6
:100A90008D3241F0830F8A3319F480E331E001C0D5
:100AA00033278C93AE1789F7332341F0AE2FBF2F36
:100AB000B8DF81E34D3209F43196808308958827A9
:100AC000E00DF81FE00FF81F80830895040F151F35
:100AD000261F371F0895000F111F221F331F08956F
:100AE00000951095209530950F5F1F4F2F4F3F4F6A
:100AF0000895019110810EC00191119121913081D1
:100B00000BC00191108117FF05C03FEF2FEF04C00C
:100B1000008111272227332737FF03C0E1DF8DE251
:100B20008D93CF93DF93CF92DF92EF92AA24BB24D1
:100B3000CC24DD24EE2440E2CAE0DD2755E093E337
:100B40008881890F87FD9F7083FD907F891B899322
:100B50005A95A9F7C0DFAA1CBB1CCC1CDD1CEE1CDF
:100B60004A9551F7E894EFE0FF2782910ED0EB30E1
:100B7000E0F71EF068948A2D0CD088278D93EF90B3
:100B8000DF90CF90DF91CF910895982F829501D07B
:100B9000892F8F70805D26F0803309F40895689462
:100BA0008D93089581918D938823E1F7089594E0C2
:100BB00081918D939A95E1F708950000A842000075
:100BC00008426D3136382D746573742D6361706120
:100BD0006369746F722D72632D74696D696E672D10
:100BE0006469726563742E762E30322E62617300F2
:100BF000636E74207065722070657263656E742018
:100C00003D20000020326176673D0000206176675C
:040C1000253D00007E
:00000001FF
